:1000000000308A00992B0000B800030EB900A40B41
:100010000D281930A400A50A20140B11390E8300F5
:10002000B80E380E090009000A108A100A1182075A
:100030008734FF340A108A100A11820707340F34FC
:10004000003407340F34023407340F3404340734D7
:100050000F34083407340F34103407340F3420348D
:1000600007340F34053407340F3409340A108A106A
:100070000A1182070934023400343F30840000083A
:10008000031950280130F800F701F70B4528F80B49
:1000900044280E30F700F70B4B280000800B422855
:1000A00000348501860118306500FF306600831634
:1000B00081138312BE2BF701F8013A0803103B1895
:1000C000F707F70CF80CBB18F707F70CF80C3B19FF
:1000D000F707F70CF80CBB19F707F70CF80C3B1AED
:1000E000F707F70CF80CBB1AF707F70CF80C3B1BDB
:1000F000F707F70CF80CBB1BF707F70CF80C0034EC
:100100000608A300FF30A3062308F839A700A70CB0
:10011000A70CA70C1F30A705271E90280310A70DBA
:100120002708BA000330BB005B207808A70023082B
:100130000739AD003C30B4002D08043C031CA52851
:100140000530AE0001302D07B0002D08053C031D21
:10015000AE280130AE00B0017830B4002D08053C67
:100160000318BB282D08073C031CBB280230AE0037
:1001700005302D02B000BF2BF801F901F701FA019B
:100180004208031DC62841080319E0281030C300A7
:100190000310BF0DC00DF70DFA0D42087A02031DC2
:1001A000D32841087702031CDC284108F702031C0E
:1001B000FA034208FA020314F80DF90DC30BC8281C
:1001C000000000341930A400A501A6010130AF00E1
:1001D0002015FF30B600003401303402B300023085
:1001E000C0005830BF00C2013408C100BC207808EC
:1001F000B700E220A8010130B10081010630F7000C
:10020000F71D0A2907308101813084000008C039B8
:100210000F3880006400813084000008C039770402
:1002200080008B16C0308B04C02B34082502031CC1
:1002300024293408A502A60AAF0A2F082E020318A3
:1002400023290130AF00201537082602031C2C2972
:10025000A601A808031DA80300341030F700FA0116
:10026000C501C20CC10C031C3B294308FA07031843
:10027000C50A4408C507C50CFA0CF90CF80CF70BB5
:100280003129003425083602031C71290330C000CF
:10029000E830BF00C2012A08C100BC207908C000B4
:1002A0007808BF007908C2007808C100C4013E0880
:1002B000C3002D217908AC007808AB002C08FA00A7
:1002C0002B080319AC03AB03BF007A08C000BF08BA
:1002D000031D6D29C008031971290130BF003D209D
:1002E0005E29003425083602031CA4290330C0000F
:1002F000E830BF00C2012A08C100BC207908C00054
:100300007808BF007908C2007808C100C4013E081F
:10031000C3002D217908AC007808AB0005188514BE
:100320002C08FA002B080319AC03AB03BF007A08B2
:10033000C000BF08031D9F29C0080319A32901306D
:10034000BF003D20902985100034BD08031DAB2956
:100350000530BE0042213D08803C0318BE293D08FF
:10036000013C0318BE290310BD0C031CBA292A083E
:10037000BE0072210130BE004221AF293D08013C80
:100380000318D4290310BD0C031CCD290330BE0073
:1003900072210130BE004221D3290130BE007221FA
:1003A0000130BE004221BE290230BE00422100348D
:1003B0000730BE004221A101210883169B009C1337
:1003C0001C141A08FF3C0319F32983122108831611
:1003D0009B009C131C141A088312BA00BD00A521AF
:1003E000A10ADC298316831200340930AA000514FF
:1003F0000730BE0042212230BD00A521D8210510C2
:10040000A10105158519022A05110608FF3AA30066
:100410002308013A0319132A813A03194F2A7F3A14
:1004200003198C2AA52AA2012208023C031C4E2A89
:1004300022083620BA00210883169B0083123A084E
:1004400083169A001C1583120B08F7008B13831672
:1004500055309D00AA309D009C149C182D2A1C111B
:10046000770883128B0401302107BA0083169B00A2
:10047000FF309A001C1583120B08F7008B138316AC
:1004800055309D00AA309D009C149C18452A1C11D3
:10049000770883128B04A10AA20A142AD62AA20181
:1004A00022081420FF3C03198B2A22081420BA00CA
:1004B000210883169B0083123A0883169A001C15A4
:1004C00083120B08F7008B13831655309D00AA305A
:1004D0009D009C149C186A2A1C11770883128B04B7
:1004E00001302107BA0083169B00FF309A001C15CB
:1004F00083120B08F7008B13831655309D00AA302A
:100500009D009C149C18822A1C11770883128B046E
:10051000A20AA10A502AD62A210883169B00831218
:10052000230883169A001C1583120B08F7008B13FF
:10053000831655309D00AA309D009C149C189E2A5D
:100540001C11770883128B04D62A210883169B007E
:100550008312230883169A001C1583120B08F700D8
:100560008B13831655309D00AA309D009C149C1857
:10057000B72A1C11770883128B0401302107BA00B7
:1005800083169B00FF309A001C1583120B08F7009E
:100590008B13831655309D00AA309D009C149C1827
:1005A000CF2A1C11770883128B04A10A0514D821C5
:1005B0000510230F012AD02B85100510A014A018B8
:1005C000E32A0511E42A0515851DE42AE2202708FF
:1005D000A8003008B100A015CF2BA80803192E2BB6
:1005E0001930AA001521003020180130013C031DEC
:1005F000012B0230A006A018FF2A0511002B0515BB
:100600002010A80803192B2B2808063C031C2B2BB1
:100610002708280203182B2B30082F02031D2B2B31
:10062000A508031D2B2B851005140730BE004221A1
:10063000A1012108023C031C2A2B3008BA00033018
:10064000BB005B20210878071A20BC00BD00A52153
:10065000A10A192B0510A808031DF22A0511D02B99
:10066000E22015212F0831020319392BB108031D8F
:10067000972B003020190130013C031D972B85106A
:1006800005140030201A0130003A031D612B193087
:10069000AA002508A20083169B019C131C141A08AB
:1006A000FF3C0319592B8312D8210330BE0042218D
:1006B0008316831222083307F80025087802B20057
:1006C00020160930AA003208B600320825020318A5
:1006D0007F2B0730BE004221A1012108023C031CF0
:1006E0007E2B3008BA000330BB005B20210878075E
:1006F0001A20BC00BD00A521A10A6D2B652B193065
:10070000AA003408B60083169B019C131C141A0817
:10071000FF3C03198E2B8312D821831683123308D2
:1007200025020318952B83168E2B05102011312BD3
:10073000D12B84011F30830507309F002010A010AB
:100740002011A0112012A101A201A301A401A50161
:10075000A601A701A801A901AA01AB01AC01AD0145
:10076000AE01AF01B001B101B201B301B401B501F5
:10077000B601B7010130BF003D2051288028EC2888
:100780008519D02B2508023C031CCA2B8519CA2BBE
:100790001521C22B851DCE2B051AF529DC2AED2A41
:0407A000302B630097
:0A42000006000A0009001400FF0088
:02400E00613F10
:00000001FF
